:10000000B6017829A4003A0884003808C92084136E
:1000100000052C1C3806031920282408031D182865
:100020002A08FF3E031C21280A30EA202A0821283A
:10003000240AFF3003192028240B20282B0821280C
:10004000AD09AD0C73290408A7008611051205122D
:100050008316861105120512F030850583122708D4
:10006000B61850283A30A1009830F8203330A60056
:1000700065201330A1008830F82065206430F72017
:1000800065206430F7202230A600652028304F20FC
:100090000C304F2006304F20B61427085028361455
:1000A000A600361C5E280512033C031C632863204F
:1000B0000730A100D030F820031408003614FE3CAD
:1000C000031973290516A60E361C36108615F03056
:1000D000850526080F3985048611A60E3618652871
:1000E0003230F72003140800B71329080319B71793
:1000F0000530A8002730A30010308A200330A30069
:10010000E8308A20A30164308A20A3010A308A20C3
:1001100024089128A2002508A1002408A0003C2161
:100120002008A000A8030319B713290803199B2866
:100130002802031808002008031DB713B71B080086
:10014000303E6E29A3003A0884003809CC2084137D
:10015000A30803197329F030A50022088038A400F1
:10016000F030A5030319A5000319A303031973298C
:10017000B928CF20030120183808A21F3808A20888
:1001800003190301A40FC6288006AD28C728000064
:10019000B0288417800473298417800573292108E7
:1001A00020040319A00A8030201AA1062019A106F4
:1001B000A018A106210DA00DA10D732983169A0088
:1001C0001C1555309D00AA309D009C149C18E628F3
:1001D0001C117329A301A200FF30A207031CA3076F
:1001E000031C73290330A100DF30F820EC28A101A3
:1001F000E83EA000A109FC30031C0129A007031858
:10020000FE28A0076400A10FFE2820180729A01CC3
:100210000B2900000B29080022211029A3011D2110
:10022000031916292308A1002208A00020080800AD
:10023000A20002302529A101A301A2000130252935
:10024000A101A301A20004302529A800230821024E
:10025000031D2C2922082002043003180130031941
:1002600002302805031DFF3073290038031DFF30BD
:100270000405031DFF307329A501A4011030A60059
:10028000210DA40DA50D2208A4022308031C230F91
:10029000A502031852292208A40723080318230FD4
:1002A000A5070310A00DA10DA60B40292008732956
:1002B0001030A800A101A001A70CA60C031C662900
:1002C0002208A00723080318230FA107A10CA00CE4
:1002D000A50CA40CA80B5C29240873298400310800
:1002E0008A0030088200831303138312640008001D
:1002F0008A11352B6030DB00932108001830DB00B9
:10030000BD21BD21BD21BD21BD218629DB0B802959
:1003100008003030DB009321CC0D08001830DB00E2
:100320009321CC0D08008617BD2186139729BD2186
:100330009929BD21BD21DB0B93290800FF30D8008E
:10034000BD21A229851A0800D80BA029A8290800D8
:100350000130D8000800FA30D800851EB429BD212C
:100360000000D80BAD29BC29FF30D800BD21B82929
:10037000851A0800D80BB6295F14080083161C14D0
:100380008312080083161C158B1355309D00AA306C
:100390009D009C148312080050106400C830EA00CD
:1003A000851ED729EA0BD029EC0BCD290800501463
:1003B00008006108053C8A11031CE82901308A0005
:1003C00061088207F6296C2A7D2A8A2A9E2AB22A87
:1003D00064006108113C8A150319E12D640061086D
:1003E000123C8A110319402B8A111B2CC901E6010A
:1003F0000330D6006400153056028A1103180D2A06
:100400008A1585245608A03E84004C0880004C08BC
:10041000C907D60A8A11031DFA298A1585246400A2
:1004200049084C028A11031D422AFE308A01242009
:1004300001308A012420FE308A01242080308A0184
:10044000242043308A0124206C308A0124206F301C
:100450008A0124206E308A01242065308A012420FC
:1004600020308A0124204F308A0124204B308A0119
:1004700024200130A300F4308A01EB208A1569277B
:100480008A15C02BFE308A01242001308A012420E5
:10049000FE308A01242080308A01242045308A01E0
:1004A000242072308A01242072308A0124206F3087
:1004B0008A01242072308A0124200616831606122F
:1004C00083120330A300E8308A01EB200612831662
:1004D000061283128A111B2C6430A000A1014C0863
:1004E0008A010E21B2002108B3003208BC0733088C
:1004F0000318013EBD078A11C22A6230A000A10183
:100500004C088A010E21B2002108B3003208E3072B
:100510008A11C22A6230A000A1014C088A010E2172
:10052000B2002108B3003208CA07831607309B00C7
:1005300083124A088A01DE208A11C22A6230A00092
:10054000A1014C088A010E21B2002108B300320833
:10055000E20783160B309B00831262088A01DE20BB
:100560008A11C22A1F304C05CB004B08A600A701F8
:100570000230A200A3018A015821CB008A15D4249D
:100580008A111B2CFA308A01EA208A1564258A1503
:1005900077278A111B2C6508A000A1012030A2003A
:1005A000A3018A013C21E6006608073C8A11031C6E
:1005B000E52A02308A0066088207E52AEF2AF92A2E
:1005C000032B0D2B172B212B2B2B53308A0124208F
:1005D00079308A01242073308A01242008005230A7
:1005E0008A01242065308A01242064308A01242075
:1005F000080042308A0124206C308A0124207530A2
:100600008A012420080059308A01242065308A019B
:1006100024206C308A012420080047308A012420DD
:1006200072308A0124206E308A0124200800423072
:100630008A0124206C308A0124206B308A01242016
:10064000080057308A01242068308A012420743041
:100650008A012420080050308A01242075308A0144
:10066000242072308A012420080007309F0083165E
:100670007F3081002130850007308600831286019B
:10068000E6016400203066028A110318522B6608C6
:10069000203E84008317003080008313E60A8A110D
:1006A000031D412BD6016400153056028A11031830
:1006B0006A2B560883169B0083128A01BE215608B6
:1006C000A03E840083161A0880008312D60A8A117D
:1006D000031D532B8316200C831203185F15031C74
:1006E0005F11831621088312DD008316220883120E
:1006F000DC00831623088312CF008316260883129A
:10070000CA0083162B0C83120318DF14031CDF109E
:1007100083162C088312D70083162D0C831203181E
:100720006014031C601083162F088312E2008316E6
:10073000300C83120318DF16031CDF128316310CF2
:1007400083120318DF17031CDF138316320C831286
:100750000318E014031CE0108316330C83120318F3
:10076000DF15031CDF115D08E5005C08E100643063
:100770004F07BC00BD01BD0D5E30BE000130BF00A3
:10078000831627088312E300C601C701C801FE30A3
:100790008A01242001308A012420FE308A0124208D
:1007A00080308A0124204D308A01242069308A015A
:1007B00024206C308A01242065308A012420733083
:1007C0008A01242054308A01242061308A012420A7
:1007D00067308A012420FE308A012420C0308A013B
:1007E000242056308A01242065308A01242072306A
:1007F0008A01242020308A01242033308A012420D9
:100800002E308A01242031308A01242035308A019B
:1008100024200330A300E8308A01EB20831605145E
:1008200064008A11831205181A2C6430BC00BD01C3
:100830008A113D2F5F128A156425C8308A01EA208B
:1008400064008A11851A262C8A118A260630BA007D
:100850000130B800AC01831628088312AA000430C6
:10086000AB000130AD0046088A010220C6008A11A3
:100870000318CB2D0630BA000430B800AC01FF30AD
:10088000AA000A30AB000130AD0047088A010220FF
:10089000C7008A110318602C0630BA000230B80075
:1008A000AC01FF30AA000A30AB000130AD004808AF
:1008B0008A010220C8008A1103181A2E8A01202CEE
:1008C00064008A11601CD32CFE308A012420013080
:1008D0008A012420FE308A01242081308A012420CC
:1008E00052308A01242050308A01242047308A0166
:1008F0002420FE308A01242085308A012420A90189
:100900006208A400A5012330B000B1018A0174205F
:10091000C8308A01EA2064008A11851A912C8A1154
:100920008A260630BA000130B800AC01FF30AA00B8
:100930000A30AB000130AD0046088A010220C60033
:100940008A110318F42D0630BA000430B800AC0147
:10095000FF30AA000A30AB000130AD0047088A0121
:100960000220C7008A110318D32C0630BA000230C7
:10097000B800AC01FF30AA000A30AB000130AD0076
:1009800048088A010220C8008A110318C92C8A016C
:100990008B2C2030860683168612FA3083128A0149
:1009A000EA208A018B2C64008A11DF1F5F2D64000E
:1009B0008A11DF185F2DFE308A01242001308A0160
:1009C0002420FE308A01242080308A0124205230E5
:1009D0008A01242065308A01242073308A01242072
:1009E00074308A01242061308A01242072308A0107
:1009F000242074308A012420FE308A012420C03053
:100A00008A01242050308A0124206C308A0124205D
:100A100061308A01242079308A01242065308A01DE
:100A2000242072308A012420C8308A01EA20640020
:100A30008A11851A1D2D8A118A260630BA000130C6
:100A4000B800AC01FF30AA000A30AB000130AD00A5
:100A500046088A010220C6008A110318122E0630A9
:100A6000BA000430B800AC01FF30AA000A30AB0075
:100A70000130AD0047088A010220C7008A1103181F
:100A80005F2D0630BA000230B800AC01FF30AA007A
:100A90000A30AB000130AD0048088A010220C800CE
:100AA0008A110318552D8A01172D203086068316CA
:100AB0008612FA3083128A01EA208A01172D8316E2
:100AC000051464008A118312051C1B2CFE308A0158
:100AD000242001308A012420FE308A012420813024
:100AE0008A01242043308A0124206F308A01242087
:100AF0006E308A01242066308A01242069308A0100
:100B0000242067308A012420C8308A01EA20063078
:100B1000BA000130B800AC01FF30AA000A30AB00C7
:100B20000130AD0046088A010220C6008A11031870
:100B30004C2F0630BA000430B800AC01FF30AA00D8
:100B40000A30AB000130AD0047088A010220C7001F
:100B50008A1103181B2C0630BA000230B800AC0111
:100B6000FF30AA000A30AB000130AD0048088A010E
:100B70000220C8008A110318BF2D8A01872D20305A
:100B800086068316861283120130A3002C308A0158
:100B9000EB208A01872D64008A115F1A202C6400E3
:100BA0006308003C8A150319BC2C831625088312A0
:100BB000C4008A15DD2364006308FB3C8A11031915
:100BC000E22DE3038A15D025831629088312EC0051
:100BD0008A01CC2164005008003C8A110319F22DCF
:100BE0008A118A268A01202C64008A115F1A1D2C22
:100BF00064006208003C8A150319BC2C83162E0879
:100C00008312C4008A15DD2364006208633C8A11E4
:100C100003190B2EE2038A156425C8308A01EA20E5
:100C20008A011D2CC4018A15DD23C8308A01EA20FF
:100C30008A01172D6400013063028A110318802E87
:100C400064004A08003C8A150319BC2C64004A0859
:100C5000633C8A1103192D2ECA03FE308A01242019
:100C600001308A012420FE308A01242081308A014B
:100C7000242052308A01242065308A0124206C30DF
:100C80008A0124206F308A01242061308A012420C7
:100C900064308A012420FE308A012420C0308A0179
:100CA00024200130E8006400093068028A1103182A
:100CB0007A2EFF308A0124200130E900640069089F
:100CC00083162A028A118312031C762E6430EC00EC
:100CD0008A01CC2164005008003C8A110319722E4D
:100CE0008A118A26E90A8A11031D5E2EE80A8A11F2
:100CF000031D532E831627088312E3008A011B2C41
:100D00002030860683168612C83083128A01EA20B4
:100D10008A011D2C5F10DE018A019E215808FF3CCC
:100D2000E6006400CE3066028A110318982E08008F
:100D30006400F63066028A110318D82E8A154424FE
:100D400064008A115F18D82E4C08CD008A154424FF
:100D500064008A115F18D82E8A01AB2164008A11C1
:100D60005F18D82E5808FF3CE600640097306602F2
:100D70008A110318D82E64001E3066028A11031CE3
:100D8000D82E6400593066028A11031CC82EDE0A70
:100D900064008A115E18D22E64008A115F1DE82E4D
:100DA0008A11D82E64008A115F19E82E8A11D82E74
:100DB00064008A115F1A3D2F061683160612FA3058
:100DC00083128A01EA200612831606128312080093
:100DD000E0304D05E5001F304D05E1006400650879
:100DE000003C8A110319D92964008A11DF18042FE5
:100DF000640065085D028A110319D82E64004C084E
:100E0000003C8A1103192D2F64008A115F1A3D2FAF
:100E10006400C9304C028A1103183B2F640065300E
:100E20004C028A110318D82E4C08CB006108203ED2
:100E3000840083170008B200831301303207B20028
:100E4000B301B30D6108203E84008317320880008F
:100E500083138A15D4248A011B2C5F120612831671
:100E60000612643083124F07BC00BD01BD0D8A1508
:100E700069278A01522B8A01D82E5F16061683161F
:100E8000061283128A15642564008A11851A4A2F76
:100E90008A018A268A01442FFE308A0124200130EB
:100EA0008A012420FE308A01242080308A012420F7
:100EB00047308A01242061308A0124206D308A0164
:100EC000242065308A01242064008A115F1D732F5D
:100ED000FE308A012420C0308A01242042308A0159
:100EE00024208A117C2FFE308A012420C0308A0100
:100EF000242041308A012420C8308A01EA200630AB
:100F0000BA000130B800AC01FF30AA000A30AB00D3
:100F10000130AD0046088A010220C6008A1103187C
:100F2000A52F0630BA000430B800AC01FF30AA008B
:100F30000A30AB000130AD0047088A010220C7002B
:100F40008A110318B52F8A017F2F64008A115F1957
:100F5000AC2F5F158A11AD2F5F1100305F19013082
:100F60008316A00083128A01642FFE308A01242098
:100F700080308A01242054308A01242065308A017F
:100F8000242061308A0124206D308A0124205D08EC
:100F9000E500FE308A012420C0308A0124208A0125
:100FA000CB22C8308A01EA200630BA000130B800EE
:100FB000AC01FF30AA000A30AB000130AD0046089A
:100FC0008A010220C6008A110318FA2F0630BA00DF
:100FD0000430B800AC01FF30AA000A30AB00013089
:100FE000AD0047088A010220C7008A15031812289D
:100FF0008A01D42F20305D07C200C301C30D42080F
:10100000A0004308A100A301F4308A011D218A1524
:10101000031D0E284208DD008A01C72F2030DD00A5
:101020008A01C72F5D088316A10083120230D60003
:10103000D4011F30D3000130D500FE308A012420B6
:1010400080308A01242050308A0124206C308A01AB
:10105000242061308A01242079308A0124206530DF
:101060008A01242072308A0124208A1553265608CA
:10107000A03E84000008E1001330D600FE308A0153
:10108000242080308A01242047308A0124202D30FA
:101090008A0124204D308A0124206F308A012420C7
:1010A00064308A01242065308A0124208A15D126E3
:1010B0005608A03E84000018DF15001CDF116400F4
:1010C0008A15DF1D87281430D6000230D400143072
:1010D000D3000130D500FE308A01242080308A01FF
:1010E000242047308A0124202D308A0124205430C6
:1010F0008A01242061308A01242067308A0124205B
:1011000073308A0124208A1553268A15FE2803305D
:10111000D6000530D40064303E02D3000530D5003F
:10112000FE308A01242080308A01242048308A0140
:10113000242065308A01242061308A0124206C300B
:101140008A01242074308A01242068308A012420F6
:101150008A1553265608A03E84000008CF000C30A4
:10116000D600D4011E30D3000130D500FE308A01F4
:10117000242080308A0124204B308A0124206530CD
:101180008A01242076308A0124206C308A012420B0
:1011900061308A01242072308A0124208A15532666
:1011A0005608A03E84000008D7000530D600013064
:1011B000D4006430D3000130D500FE308A012420F1
:1011C00080308A01242047308A01242075308A012A
:1011D00024206E308A01242020308A0124204830C7
:1011E0008A01242050308A0124208A15532656086B
:1011F000A03E840000088316A50083120630D600A6
:101200000130D4006330D3000130D500FE308A01B4
:10121000242080308A01242043308A0124206C302D
:101220008A01242069308A01242070308A01242018
:1012300073308A01242020308A0124208A15532605
:101240005608A03E84000008CA000730D6000130CE
:10125000D400FB30D3000130D500FE308A012420B9
:1012600080308A01242052308A0124206F308A0184
:10127000242075308A0124206E308A0124206430B5
:101280008A01242073308A0124208A1553265608A7
:10129000A03E840000088316A700831264008A150C
:1012A000DF1D552960108A15CC290D30D600FE307F
:1012B0008A01242080308A01242052308A0124208F
:1012C00050308A01242047308A01242020308A01AE
:1012D000242020308A01242020308A0124208A15ED
:1012E000D1265608A03E840000186014001C60102F
:1012F00064008A15601CCC290E30D6000530D4005D
:10130000C830D3000530D500FE308A01242080305B
:101310008A01242052308A01242050308A0124205E
:1013200047308A01242020308A01242048308A0155
:10133000242050308A0124208A1553265608A03EC6
:10134000840000088316AE0083120F30D6000130EF
:10135000D4006330D3000130D500FE308A01242050
:1013600080308A01242052308A01242050308A01A2
:10137000242047308A01242073308A012420203021
:101380008A01242020308A0124208A1553265608F9
:10139000A03E84000008E2000830D60064008316F6
:1013A0002808FF3C8A158312031DDD295608A03E3C
:1013B0008400003080008A15E2295608A03E84008F
:1013C00001308000FE308A01242080308A012420F0
:1013D00046308A0124202D308A01242041308A01A0
:1013E000242075308A01242074308A0124206F3033
:1013F0008A0124208A15D1265608A03E84000008C0
:10140000B20064003208003C8A15031D0D2A8316C1
:10141000FF30A80083128A15112A83160130A80014
:1014200083120430D600D4011430D3000130D5002B
:10143000FE308A01242080308A01242048308A012D
:10144000242069308A01242074308A012420443009
:101450008A0124206C308A01242079308A012420DA
:101460008A1553265608A03E840000088316A4005F
:1014700083120930D6000A30D400C830D3000530BA
:10148000D500FE308A01242080308A012420433098
:101490008A01242079308A01242063308A012420A3
:1014A0006C308A01242069308A01242063308A014B
:1014B00024208A1553265608A03E8400000883166F
:1014C000A90083120A30D6000130D4001E30D300A8
:1014D0000130D500FE308A01242080308A0124208A
:1014E00052308A01242065308A0124206C308A0120
:1014F00024206F308A01242061308A012420643046
:101500008A0124208A1553265608A03E840000082C
:101510008316AA0083121030D600FE308A012420E0
:1015200080308A0124204D308A01242075308A01C0
:1015300024207A308A0124207A308A0124206C30D9
:101540008A01242065308A0124208A15D126560874
:10155000A03E84000018DF16001CDF121130D600F8
:10156000FE308A01242080308A01242052308A01F2
:10157000242065308A01242073308A0124207430AD
:101580008A01242072308A01242074308A012420A8
:101590008A15D1265608A03E84000018DF17001CCB
:1015A000DF131230D600FE308A01242080308A01F9
:1015B000242053308A0124206F308A012420753082
:1015C0008A0124206E308A01242064308A0124207C
:1015D00020308A0124208A15D1265608A03E840096
:1015E0000018E014001CE0100B30D600FE308A0119
:1015F000242080308A01242046308A012420723041
:101600008A01242046308A01242069308A0124205E
:1016100072308A01242065308A0124208A15D1265F
:101620005608A03E84000018E014001CE010FE30B4
:101630008A01242001308A012420FE308A012420DE
:1016400080308A01242043308A0124206C308A01B2
:1016500024206F308A0124206E308A0124206530D6
:101660008A01242020308A012420C8308A01EA20FF
:101670000630BA000130B800AC01FF30AA000A30D1
:10168000AB000130AD0046088A010220C6008A1571
:1016900003185E2B0630BA000430B800AC01FF30EE
:1016A000AA000A30AB000130AD0047088A010220D1
:1016B000C7008A1503187F2B8A15382BC901DA0158
:1016C0008A15E2230330D6006400153056028A15CD
:1016D0000318772B5608A03E84000008CC004C0865
:1016E000C9078A152A24D60A8A15031D642B4908BE
:1016F000CC008A152A248A1585278A15172BFE30D7
:101700008A01242080308A01242053308A01242039
:1017100061308A01242076308A01242065308A01D4
:10172000242020308A0124203F308A012420C83020
:101730008A01EA200630BA000130B800AC01FF305F
:10174000AA000A30AB000130AD0046088A01022031
:10175000C6008A150318C02B0630BA000430B80042
:10176000AC01FF30AA000A30AB000130AD004708E1
:101770008A010220C7008A1103184C2F8A159A2B60
:10178000D6016400143056028A150318DB2B560864
:1017900083169B0083125608A03E8400000883161F
:1017A0009A0083128A01C22132308A01EA20D60AC5
:1017B0008A15031DC12B8A01522B5C085D04CC00E5
:1017C0008A15E42B5A08CC00DE018A017A218A1599
:1017D0002A244408CC008A152A248A017E21640028
:1017E0008A155F19FF2B64008A155E1CFB2B8A018A
:1017F00089218A15FD2B8A018E218A150B2C640004
:101800008A155E1C072C8A018E218A15092C8A01F3
:1018100089218A150B2C64008A15E01C132C0616EE
:1018200083160612831264008A15DF1E1B2C06170E
:1018300083160613831219308A01EA2006128316D2
:1018400006128312061383160613013083128A01CF
:10185000EA2008000130C5006400093045028A15FD
:101860000318432C8A017E2164008A15CC1B3C2C72
:101870008A018E218A153F2CDE0A8A018921C50A38
:101880008A15031D2C2C08000130C50064000930A6
:1018900045028A150318842C4C08A600A7010230C3
:1018A000A200A3018A015821CC008A01AB21640067
:1018B0008A155F1C5C2C08005808FF3CE60066088F
:1018C000A00096308A012021B2006608A0001E30D8
:1018D0008A011B21B4003208840034088A013521B2
:1018E0008A15031D752C5F140800640059306602C8
:1018F0008A1503187E2C4C108A15802CDE0A4C1495
:10190000C50A8A15031D462C0800851A852C01304E
:10191000C5006400093045028A150318BB2C4C0829
:10192000A600A7010230A200A3018A015821CC0021
:101930008A01AB2164008A115F18422A5808FF3CD3
:10194000E6006400973066028A110318422A640098
:101950001E3066028A11031C422A64005930660256
:101960008A150318B62C4C108A15B72C4C14C50ACE
:101970008A15031D892C080064008A11E01C1B2CA9
:101980000630BA001030B8006430A2000A308A0174
:10199000A2203230A2000A308A01A2200612831649
:1019A000061283128A011B2C6108203E84008317D3
:1019B0000008B200831301303207B200B301B30D47
:1019C0006108203E8400831732088000831364007E
:1019D0008A15DF1DFC2C6108203E84008317000857
:1019E000B200831364003208831634028A11831212
:1019F00003193D2F8A15222D64005708003C8A15D3
:101A00000319052D0310CB0CD7034B083C02B20081
:101A10003D08031CFF3EB3006430A000A101330861
:101A2000A30032088A010C21BC002108BD003C083B
:101A3000A0003D08A100A30164308A0118218A1189
:101A4000031D3D2F8A155B278A15642564008316C4
:101A50002408003C8A1583120319632D8616831609
:101A60008612FE3083128A01242001308A0124204C
:101A7000FE308A01242082308A01242057308A01D6
:101A8000242041308A01242049308A012420543006
:101A90008A012420E830A6000330A700831624081A
:101AA0008312A200A3018A015821C0002508C100A9
:101AB0004108A30040088A01EB2086128316861293
:101AC00083128A011B2C0800FE308A012420013079
:101AD0008A012420FE308A01242080308A012420BB
:101AE00052308A0124200330A9006308A400A50114
:101AF0002330B000B1018A017420FE308A01242015
:101B000085308A01242043308A0124200230A90034
:101B10004A08A400A5012330B000B1018A01742055
:101B200064303C02E60064008A15DF1DB32DFE30F0
:101B30008A012420C0308A01242054308A012420C4
:101B40000230A9006108203E840083170008B2001B
:101B500083133208A400A5012330B000B1018A012B
:101B600074208A15C32DFE308A012420C0308A01DA
:101B700024200330A9006608A400A5012330B0008A
:101B8000B1018A0174208A01CB220230A9006108C8
:101B9000A400A5012330B000B1018A01742008001F
:101BA000FE308A01242081308A0124200330A900DC
:101BB0006308A400A5012330B000B1018A0174209C
:101BC0000800FE308A01242001308A012420FE30E2
:101BD0008A01242080308A01242053308A01242065
:101BE00063308A0124206F308A01242072308A01F8
:101BF000242065308A01242054308A012420783042
:101C00008A012420C8308A01EA200630BA00013057
:101C1000B800AC01FF30AA000A30AB000130AD00C3
:101C200046088A010220C6008A1503182B2E0630AA
:101C3000BA000430B800AC01FF30AA000A30AB0093
:101C40000130AD0047088A010220C7008A1103183D
:101C50001B2C8A15382BC9011030DA008A15E223B3
:101C60005D085C04CC008A152A24D601640020306B
:101C700056028A1503184B2E5608203E84008317FF
:101C80000008CC0083134C08C9078A152A24D60AF9
:101C90008A15031D362E4908CC008A152A248A1578
:101CA00085278A15E12DFE308A012420C0308A0163
:101CB00024200330A9005608A03E84000008B2008A
:101CC0003208A400A5012330B000B1018A017420BC
:101CD000C8308A01EA200630BA000130B800AC01F1
:101CE0000A30AA000A30AB000130AD0046088A0174
:101CF0000220C6008A150318AE2E0630BA00043042
:101D0000B800AC01FF30AA000A30AB000130AD00D2
:101D100047088A010220C7008A150318A32E06303F
:101D2000BA000230B800AC01FF30AA000A30AB00A4
:101D30000130AD0048088A010220C8008A15031846
:101D4000A42E8A156B2E0800203086068316861274
:101D5000FA3083128A01EA208A156B2E5608A03EBB
:101D600084000008B20032085507B200B301B30D79
:101D70005608A03E8400320880005608A03E840029
:101D80000008B2006400320853028A15031CCA2EF0
:101D90008A15532E5608A03E8400540880008A15E8
:101DA000532E5608A03E84000008B200640032089A
:101DB000013C8A15031DED2EFE308A012420C0301F
:101DC0008A0124204F308A0124206E308A01242089
:101DD00020308A0124208A15FC2EFE308A0124201E
:101DE000C0308A0124204F308A01242066308A01C5
:101DF000242066308A012420C8308A01EA20063077
:101E0000BA000130B800AC01FF30AA000A30AB00C4
:101E10000130AD0046088A010220C6008A15031869
:101E2000422F0630BA000430B800AC01FF30AA00DF
:101E30000A30AB000130AD0047088A010220C7001C
:101E40008A150318372F0630BA000230B800AC01EB
:101E5000FF30AA000A30AB000130AD0048088A010B
:101E60000220C8008A150318382F8A15FF2E080093
:101E70002030860683168612FA3083128A01EA2001
:101E80008A15FF2E5608A03E84000008B2006400A8
:101E90003208013C8A15031D542F5608A03E8400C9
:101EA000003080008A15592F5608A03E840001306A
:101EB00080008A15D12E0630BA001030B8003230BA
:101EC000A2000A308A01A22006128316061283128B
:101ED00008000616831606121E3083128A01EA20B5
:101EE000061283160612323083128A01EA20061681
:101EF000831606121E3083128A01EA200612831608
:101F00000612323083128A01EA2006168316061260
:101F10001E3083128A01EA200612831606128312EB
:081F2000080063008A15912FEF
:02400E005C3F15
:104200000000200001006400020019006300140097
:10421000FF00320003000000000000002300030044
:0A422000010001000100000004008D
:00000001FF
